:100000000010001003010000D5000000D700000020
:1000100000000000000000000000000000000000E0
:10002000000000000000000000000000D9000000F7
:100030000000000000000000DB000000DD00000008
:10004000DF0000001104000031040000DF000000A8
:10005000DF000000DF000000DF000000DF00000024
:10006000DF000000DF0000000000000000000000D2
:100070000000000000000000DF000000DF000000C2
:10008000DF000000DF0000005D0D0000DF00000069
:10009000DF000000AD0C0000DF000000DF0000000A
:1000A000DF000000CD080000DF000000DF000000DE
:1000B0000000000000000000DF0000000000000061
:1000C000241A0000000000100800000008000010C2
:1000D000B4020000FEE7FEE7FEE7FEE7FEE7FEE70C
:1000E000002310B5934203D21C585C500433F9E747
:1000F00010BD00238B4203D200221A500433F9E7CB
:10010000704710B50C4C0D4B9C4206D220686168BC
:10011000A268FFF7E5FF0C34F5E7094B9C4205D2D6
:1001200020686168FFF7E5FF0834F6E700F06AFD34
:1001300001F0E8F9FEE7C046C0000000CC00000076
:10014000D4000000FFFFFFFFFFFFFFFFFFFFFFFFE7
:10015000FFFFFFFFFFFFFFFFFFFFFFFFFFFFFFFFAF
:10016000FFFFFFFFFFFFFFFFFFFFFFFFFFFFFFFF9F
:10017000FFFFFFFFFFFFFFFFFFFFFFFFFFFFFFFF8F
:10018000FFFFFFFFFFFFFFFFFFFFFFFFFFFFFFFF7F
:10019000FFFFFFFFFFFFFFFFFFFFFFFFFFFFFFFF6F
:1001A000FFFFFFFFFFFFFFFFFFFFFFFFFFFFFFFF5F
:1001B000FFFFFFFFFFFFFFFFFFFFFFFFFFFFFFFF4F
:1001C000FFFFFFFFFFFFFFFFFFFFFFFFFFFFFFFF3F
:1001D000FFFFFFFFFFFFFFFFFFFFFFFFFFFFFFFF2F
:1001E000FFFFFFFFFFFFFFFFFFFFFFFFFFFFFFFF1F
:1001F000FFFFFFFFFFFFFFFFFFFFFFFFFFFFFFFF0F
:10020000FFFFFFFFFFFFFFFFFFFFFFFFFFFFFFFFFE
:10021000FFFFFFFFFFFFFFFFFFFFFFFFFFFFFFFFEE
:10022000FFFFFFFFFFFFFFFFFFFFFFFFFFFFFFFFDE
:10023000FFFFFFFFFFFFFFFFFFFFFFFFFFFFFFFFCE
:10024000FFFFFFFFFFFFFFFFFFFFFFFFFFFFFFFFBE
:10025000FFFFFFFFFFFFFFFFFFFFFFFFFFFFFFFFAE
:10026000FFFFFFFFFFFFFFFFFFFFFFFFFFFFFFFF9E
:10027000FFFFFFFFFFFFFFFFFFFFFFFFFFFFFFFF8E
:10028000FFFFFFFFFFFFFFFFFFFFFFFFFFFFFFFF7E
:10029000FFFFFFFFFFFFFFFFFFFFFFFFFFFFFFFF6E
:1002A000FFFFFFFFFFFFFFFFFFFFFFFFFFFFFFFF5E
:1002B000FFFFFFFFFFFFFFFFFFFFFFFFFFFFFFFF4E
:1002C000FFFFFFFFFFFFFFFFFFFFFFFFFFFFFFFF3E
:1002D000FFFFFFFFFFFFFFFFFFFFFFFFFFFFFFFF2E
:1002E000FFFFFFFFFFFFFFFFFFFFFFFFFFFFFFFF1E
:1002F000FFFFFFFFFFFFFFFFFFFFFFFFFFFFFFFF0E
:100300000823802230B5041C1440651EAC4149000E
:100310000919064C5208A14202D9054C89B2614024
:10032000013B002BEFD188B230BDC046FFFF00007B
:100330002110000070B50E1C051C041C0021331B8D
:10034000EB18002B05DD2078FFF7DAFF0134011CE4
:10035000F5E70020FFF7D4FF011C0020FFF7D0FFD6
:1003600070BD000013B5154C0021201C172201237D
:1003700000F0E6FE201C00210E22022300F0E0FE29
:10038000201C00211622012300F0DAFE201C00218F
:100390001022012300F0D4FE201C00210D22022394
:1003A00000F0CEFE201C0C220223002100F0C8FE2B
:1003B0000348694600F0C8FD13BDC0460040044034
:1003C00000C0014038B5041C012210480D1C211C3E
:1003D00000F024FE0D480121002200F00BFE0B4826
:1003E000211C002200F0EBFD0128F8D12A1C211C61
:1003F000064800F0D9FD211C0448002200F00EFE42
:10040000002102480A1C00F0F5FD38BD00C0014083
:100410000223054A01211380A022D2055172002136
:100420005174024A536270470A00001000C0044031
:100430000222064B5A80A023013ADB051A720022E1
:10044000DA72034B04325A627047C0460A00001049
:1004500000C0044038B5444C0021201C1522102354
:1004600000F06EFE201C00210722102300F068FE21
:10047000201C00210622102300F062FE201C002117
:100480000922102300F05CFE201C0021082210230A
:1004900000F056FE201C00210222102300F050FE26
:1004A000201C00210322102300F04AFE201C002102
:1004B0001122102300F044FE201C00210B221123E6
:1004C00000F03EFEA02380228020DB059201995897
:1004D0008003014380209950995808240143995082
:1004E00099584038014399509958C130FF30014321
:1004F000995099580138FF380143802099509958F4
:10050000800201438020995099580001014399507D
:100510000421802598582D03884398509858A0436B
:100520009850124A5418E06F2843E067BE24022016
:10053000032564001051641815510D4A1468844352
:10054000146014688C43146050615161094A106052
:100550001160002203395A75DA719A7159725A740E
:100560001972DA7238BDC046004004400080044071
:1005700000C0044000E100E0F8B51E4B1E4A1880A0
:100580001E4B0240184012110001A023104300220C
:100590000725DB0587B29A713E1C0122A0232E415C
:1005A0000024DB051640DC715E75DA71013DF3D283
:1005B00080210901DC7139409A719C71A14204D0FB
:1005C0005C725A740E4B1A8001E05A725974A0235F
:1005D000002100B2DB050122884204DA1972DA72C6
:1005E000074B5A8001E01A72D972282000F062F994
:1005F0000020F8BD08000010F0F0FFFF0F0F000012
:100600000A000010031C0120834203D8C01A024BC9
:100610004000185C7047C0460A0000103A2330B50D
:100620008BB00093041C05A96846174B9847059D9D
:100630000120002D26D1069B201C1A0C19069BB206
:10064000090C1B0A0B43110A1206120C0A431B0465
:10065000134306A90422069300F04CFF079B201DBC
:100660001A0C19069BB2090C1B0A0B43110A12063D
:10067000120C0A431B04134307A90422079300F03A
:1006800039FF281C0BB030BDF11FFF1FA021054B07
:10069000C9051A780020002A00D10120D2434870F1
:1006A0001A7070470E000010A021054BC9051A787A
:1006B0000020002A00D10120D24308711A7070472F
:1006C0000F000010A021054BC9051A780020002A50
:1006D00000D10120D24348711A70704714000010F5
:1006E000A021054BC9051A780020002A00D101205D
:1006F000D24308701A70704715000010002138B5F9
:1007000080251D4C0A1C201C112300F019FD6D00D2
:10071000201C00210122102300F012FD201C2B1CA4
:100720000021042200F00CFD201C2B1C00210522BE
:1007300000F006FDA02480230221E4059B01E2587D
:10074000FF3D2A43E250E258FA200A43E250E258C1
:100750000E310A43E250E25810310A43E2500023BE
:100760008000237063702371637100F0A3F825701B
:1007700065702571657138BD00400440F8B545BA13
:10078000ADB2404EEBB233803F4C02232A0709D56D
:10079000FA2122680320134349003C4A236000F0F9
:1007A0003FFB09E0226803209A43226000F048FBE7
:1007B000A0230122DB055A70338801275B0709D586
:1007C000FA21236802201F434900314A276000F0C4
:1007D00027FB08E023680220BB43236000F030FBC6
:1007E000A023DB051F70A0233188DB0501228807C9
:1007F00002D50020587000E05A70114201D000224A
:1008000000E001221A7008232D0A758022681D421B
:1008100008D0FA211343052049001E4A236000F046
:10082000FFFA08E09A430520226000F009FBA023AC
:100830000122DB055A7104207388034208D0FA2193
:10084000236849000343144A236000F0E9FA08E0F2
:1008500023688343236000F0F3FAA0230122DB0521
:100860001A71A0237188DB050122880702D50020B8
:10087000587100E05A71114201D0002200E00122BB
:100880001A71F8BD10000010180000108D0600004D
:10089000E1060000C5060000A906000000230128AB
:1008A00004D80133181A9840014BC35A181C7047DA
:1008B00010000010002807D0962301385B01C046C5
:1008C000013B002BFBD1F5E77047000004210448F1
:1008D00008B503680B4201D000F038FC08BDC046E3
:1008E00000400040F0B58BB000F0C2FA00F020FCF0
:1008F00000F05CFAFFF702FFFFF734FD00F08AF921
:10090000FFF7A8FD0020B449021C00F089FAFA2183
:1009100001208900002200F083FA0024012C00D17C
:10092000D6E000F0D1F9272800D8CCE0AB4D00216B
:100930002822281C00F0E2FD281C282100F0CCF918
:100940000024061E282E00D0CAE0EB1DDF7F2B1CE2
:100950000833DB7F3F02A81D20211F43FFF7EAFC7D
:10096000874200D0AFE0201C9B49221C00F058FABF
:10097000AB78222B00D17FE02ED8102B00D0A2E044
:10098000974D211C321C281C00F0B8FDAF1D954866
:10099000FFF744FE93490822381C00F0ABFD281CE9
:1009A0000F2291490E3000F0A5FD43232B700B332D
:1009B0006B700E3BAB703F3B2B716B712021EC7069
:1009C000381CFFF7B7FCEB1D020ADA772B1C083343
:1009D000D877311C281C4CE0242B54D0302B72D1FA
:1009E0007F4D321C281C211C00F088FD2E1C7F4BE3
:1009F000E25A3319110A02349971DA710E2CF6D1C8
:100A000000240020FFF7FEFD201C2C75FFF7FAFDE7
:100A100068750120FFF7F6FD0120AC75FFF7F2FDC8
:100A2000E875201CFFF73AFF000A2876201CFFF724
:100A300035FF68760120FFF731FF000AA876012014
:100A4000FFF72CFF43232B700B336B70063BAB700F
:100A5000473BE8762B716B712021EC70B01DFFF7DE
:100A600069FCF31D020ADA77331C0833D877282192
:100A7000301C00F065F926E0A879EB7900021843F4
:100A8000FFF77AFD1FE0EB78002B06D1A879EB7910
:100A900000021843FFF772FE15E0012B13D1A8796D
:100AA000EB7900061B0418436B7A18432B7A1B0260
:100AB000184300F084FE4E4B4E4A00F065FD00F0F6
:100AC0001FFE4D4B1860002000F0C6F9041C07E023
:100AD00000F0FAF80024272383426441E4B230BFD7
:100AE000012000F0B9F9002800D117E7434E444D2A
:100AF0003188032049006918FFF764FC318806201B
:100B0000033149006918FFF75DFC31880520063183
:100B100049006918FFF756FC318805200931490062
:100B20006918FFF74FFC318801200C314900691822
:100B3000FFF748FC318802200F3149006918FFF7A0
:100B400041FC31880720123149006918FFF73AFC4F
:100B50003388281C01339BB2022B00D900230022CA
:100B60003380002303AD535104321C2AF9D10022F3
:100B7000062151439700C618715AEE59013289195E
:100B8000E951072AF4D10233062BF0D100261A4B83
:100B90001B6801937300E858032100F0BAFC00F0D1
:100BA000BDFE019900F016FE00F074FE0F4FF053E9
:100BB00002360C2EEED10321A86900F0AAFC00F049
:100BC000ADFE00F067FEFA21B88189000120002205
:100BD00000F026F9A2E6C046B80B0000760000102F
:100BE000240000101C000010AC1900009E00001032
:100BF0004D62503FFCA9F1D200000010AC00001083
:100C00004C00001008B5002000F038F900F03CF965
:100C100008BD000010B51D4C0021201C122201232C
:100C200000F08EFA201C1A4C13220123002100F040
:100C300087FA201C00F0AEFBE121201C490200F0E5
:100C40001BFC0323E3607E33A360013B2363114954
:100C500001222033104800F0B1FA10490122A023EC
:100C60000F4800F0ABFA0522C521636889001343E1
:100C70000C4A636050580C4B03408020C001034372
:100C8000535080239B03136010BDC04600400440B6
:100C900000800040AE0000105001001078010010EC
:100CA0006401001000E100E0FF00FFFF08B5034809
:100CB0000349044A00F0C9FB08BDC046008000405B
:100CC0005001001064010010024AD3681069181A1C
:100CD0007047C04650010010F0B585B002AB9D1DB5
:100CE000002302AA144ED71D01912B703B70041CE7
:100CF00001331248311C2A1C00F0A0FB2B78432B37
:100D000001D0002016E001230C48311C3A1C00F0F1
:100D100095FB3B784E2BF4D1201E0AD02A786370C5
:100D2000019B2270023BA21C0448311C00F086FB90
:100D300080B2023005B0F0BD5001001000800040CC
:100D400008B5021E04D00B1C0248034900F057FBF3
:100D500008BDC0460080004064010010022238B582
:100D60000F4B1968114219D00E4C0F4D1A60231FFA
:100D70001B78002B0FD02368002B0CD0013B236085
:100D8000002B08D1A368002B01D0984701E0012374
:100D90002373636823601434AC42E8D138BDC04685
:100DA000004001401C020010BC02001038B5184978
:100DB000184B0022181F02701A605A609A601A734A
:100DC00014338B42F5D1144C201C00F0CDF900F007
:100DD000A5F9051C201C00F0E5F90822FA21636939
:100DE000281C13436361890000F093FB1022E0612B
:100DF0006369C021134380226361084BD20249001A
:100E00005A501A60012263681343636038BDC046BC
:100E1000BC0200101C0200100040014000E100E094
:100E20001423584310B5054C133B035500232018D9
:100E300041608160C260037410BDC046180200109A
:100E400014235843034A835C002B01D000238354AE
:100E50007047C046180200101422131C4343034974
:100E6000585C002801D0CB18187C7047180200107D
:100E7000A02008B5C00500F063FA08BD014B18605A
:100E80007047C0460400001073B5202000F070FACF
:100E900000230193019BFF2B02DC019B0133F8E748
:100EA0001E4D1F4C287800F0CDF8802000F050FA3D
:100EB00023238020A36000F05BFA0123E268184E30
:100EC0001A42FAD003200221164AB36713698343FA
:100ED0000B43136100F0CAF82868C0B200F0BCF8F8
:100EE000232380203361400000F042FA6369DB076E
:100EF000FCD5802100240C4A4902D36F0B43D367F1
:100F00000A4AA300995CD3185A7809485B880134CF
:100F100000F016F9092CF3D173BDC046040000108F
:100F20000080044000C0034004800440C019000059
:100F3000004004400268034B090613401943016056
:100F40007047C046FFFFFFF838B5041C10200D1C89
:100F500000F00EFA8021104A8901D36F0B43D3674A
:100F600000230E4AE3602A602B716B7100F0D6F803
:100F700007232D7940001D4080236D049B031D43F2
:100F8000074B0849C01800F0C4FA0138C0B200028B
:100F90002843206038BDC04604800440801A060003
:100FA0008023430000478600043189000B5800204D
:100FB000834203DA1B049B0D138001307047012A22
:100FC0000ED0002A07D0022A11D1006B000C411E5E
:100FD0008841C0B20CE0006B0123C840184007E014
:100FE000006B0831C9B2C8400240D0B200E0002016
:100FF0007047000008B501290AD9002A04D08022D0
:1010000003681205134302E00268034B13400360B8
:10101000FFF790FF08BDC046FFFFFFF7012A04D18C
:101020008A4003681A43026008E00268044B1340D8
:1010300001228A4003600368934303607047C046FF
:10104000FFFFFFF80022034B18645A6401325A6410
:101050007047C046008004400022034B9864DA6465
:101060000132DA647047C046008004400022034B1E
:1010700018675A6701325A677047C04600800440BB
:1010800008B5074B596A1F23CA05120F1940054BB3
:10109000920001314900D05800F03BFA08BDC0462B
:1010A00000800440E4190000064B1A6C032313402F
:1010B00005D00020012B03D1034B186800E0034842
:1010C0007047C04600800440BC190000001BB700F8
:1010D000044B10B59C68FFF7E7FF1F232340013343
:1010E000584310BD0080044008B50A4B1A6F032313
:1010F0001340022B06D0032B07D0012B08D1FFF79A
:10110000D3FF06E0FFF7BCFF03E0FFF7E1FF00E0DD
:10111000014808BD00800440001BB70008B5FFF778
:10112000E3FF024B996F00F0F4F908BD0080044022
:1011300008B5FFF7F3FF014B186008BDB8020010B7
:10114000002900D018329200135070474B0703D586
:101150001B230268134003600822114202D0036877
:1011600013430360704700000A4A0A23904209D0E3
:10117000094A033B904205D0084BC0184342434103
:101180000920C31A01209840031C0549CA6F134364
:10119000CB6770470080014000C000400000FFBFE7
:1011A00004800440002243684260013282600132C0
:1011B00042608268002AFCD143607047436000238C
:1011C000016082600361C36001207047F8B5041CB0
:1011D000C3680768626800691B1A002093420FDA2F
:1011E0000D1CE068111C00F094F9A6687143321CD4
:1011F0007818291C00F07EF90120E3680133E360D0
:10120000F8BDF7B5036846680193C36804691C1B01
:101210000023B44236DAC36807690091041C311C0C
:10122000C068DF1B151C00F074F9F71B7B18381C15
:10123000B34200D3701A3F1A061EAE4200DD2E1CC8
:10124000AD1BBD4200DD3D1CA268019B51437243B2
:101250005818009900F04EF9E3686168F018E060F2
:1012600000F057F9A768236879435818391C3A1CCD
:101270007143009B6A43591800F03CF9E3685B191D
:10128000E3607319181CFEBDF8B5C2680369041C3D
:10129000076800209A420FD00D1C2069616800F099
:1012A00038F9A668281C7143321C791800F022F91D
:1012B0000120236901332361F8BDF7B50368C468D1
:1012C0000193036900269C4238D04668C7680369C9
:1012D0000091041C311C0069FF1A151C00F019F95B
:1012E0007B18381CB34200D3701A3F1A061EAE4258
:1012F00000DD2E1CAD1BBD4200DD3D1CA268019B24
:10130000514300987243591800F0F4F8A768236914
:10131000391C7143F018009B20615B1861680093D1
:1013200000F0F7F83A1C794323686A43591800988B
:1013300000F0E0F8236976195B192361301CFEBDCB
:101340004021024AD36F0B43D367704704800440A7
:101350008E22054992008B581843044B1840E8230D
:101360001B0218438850704700800440FF050000AE
:101370008E2110B5054C89006358054A1340024080
:101380009343E82212021343635010BD00800440CF
:10139000FF05000010B58024074B6401191DCA6FBA
:1013A00098332243CA6701221A6007238360043BF3
:1013B000C3600D33836210BD0080044037B5041C48
:1013C0000D1C6369DB0707D56A462368D11D281CFD
:1013D0000B70FFF7FBFEF4E737BD73B5051C0E1C61
:1013E0006B699B060AD56B46DC1D301C211CFFF780
:1013F0004BFF002802D023782B60F1E773BDF7B5CF
:10140000161C022201934368051C93430F1C436082
:10141000019A081C311CFFF7F4FE041C391C281C1F
:10142000FFF7DBFF019B31191A1B381CFFF7E9FEA0
:1014300002226B68001913436B60FEBD08B5081CDF
:10144000111C1A1CFFF739FF08BDF8B502264368C6
:10145000041C0D1C171C334209D0111CFFF7BDFFE3
:10146000FA683B699A4202D16368B3436360291CFE
:10147000201CFFF7A3FFF8BDF7B50D01061CFFF711
:1014800033FE291C071C00F044F800200C1E844287
:1014900006D0281C00F03DF800240C238342644150
:1014A0000F2318400190281C0199604300F031F887
:1014B0004119381C00F02DF88022F368011C1343F9
:1014C000F360FF23051C19403160010A0B40736073
:1014D000F36820019343F360019B01991B012343AF
:1014E000B362684300F015F82D014119381C00F073
:1014F00010F8FEBD08B500F02EFA08BD08B500F0E2
:1015000040FA08BD08B5FFF7EDF908BD03000B432D
:1015100021D4002931D00122D207030901E00901B9
:1015200012099942FBD9430801E049005208994247
:10153000FBD900E04908401A07D35241FAD30146CB
:101540001046704749084018F7D29218FAD340184D
:10155000014610467047CB0F00D04942021000D51B
:101560004042534008B5FFF7D4FF0CBC521000D3E3
:101570004042002A00D549421847F446002000F0B6
:1015800001F8604770470000F0B5071C081C4D00CB
:1015900087B06D0D5840002D7DD0504CA5427AD0BB
:1015A0005E00760D77D0A64275D0141C7219802586
:1015B00009038026090B6D030D430021C00F019222
:1015C000C2070092DB02620D134336061E432A1C3B
:1015D000301C0B1C00F0A8F9029003910021E402DA
:1015E000221C281C0B1C00F09FF9059100213A1CBD
:1015F00004900B1C301C00F097F90E1C00213A1CC3
:10160000051C0B1C201C00F08FF98446081C0021CF
:101610000B1C049A0F1C12184B41521973411E1CCB
:101620000B1C02980399141C059A92197B411218FD
:101630004B41614688080443019929480918294803
:1016400098420CD3161C1F1CB6185F4126483B1C41
:101650008446E00F3043021C019964006144002776
:10166000E60F92197B418020151C0006844201D1AF
:10167000012085431D48814205D80A050099281C90
:101680001943511827E0009B002902DB184B009AF0
:10169000134300201EE0C20F1648D20749008142C2
:1016A00005D85C00844205D80020111C13E01248C4
:1016B000814203D110485B00834201D9002005E03C
:1016C000490D0020002901D05B0D01D10B4902E03A
:1016D000074B1343191C07B0F0BDC046FF070000BD
:1016E00001FCFFFFFFFF0F0000FCFFFFFD070000F4
:1016F0000000F07FFFFFDFFF0000E0FF0000F87F49
:1017000030B5021C124CC80F4900C307114D4808E0
:101710000419AC420FD8C82424060019D100C00017
:10172000520F0243C80F10188022120691420AD1AC
:101730000122904307E0181C002C07DB064A914267
:1017400003D8FF20C005184300E0044830BDC04660
:101750000000F0C7FFFFDF0F0000E0FF0000C07FC8
:1017600010B5002802D1031C021C25E0030C01D196
:10177000000402E080235B04C918030E01D10002BB
:1017800002E080231B04C918030F01D1000102E00D
:101790008023DB03C918830F01D1800002E080237E
:1017A0009B03C918002801DB400002E080235B0393
:1017B000C918C41263184205101C191C10BDC10FB2
:1017C00008B5C90700D040428023DB05C918FFF7E0
:1017D000C7FF08BD70B5C50DFF232A1C0C1C1A409D
:1017E0004440002A33D09A4231D0CD0D1D402ED036
:1017F0009D422CD055198022090212060002104386
:101800000A4300210B1C00F08FF80E1E01DA7F3D09
:1018100001E0803D4E00E40F330AE407EA0523436C
:101820009B18802236061206964204D0FD2D02D85F
:10183000F60F981929E00133002801D101229343C2
:10184000181CFD2D21D9201C002D19DA1DE00F4B8D
:101850004000984205D84A009A4206D8E00FC007D7
:1018600013E0FF231B0698420ED1FF2349001B06FD
:10187000994209D8000E07D0090E05D0E40FE407FD
:10188000FF20C005204300E0014870BDFFFFFFFEC0
:101890000000C07F10B580249E23C10D02022406E3
:1018A00022435B1A02D4DA40101C06E0FE2902D95A
:1018B0000020A24201D1090A481E10BD00282BD0E9
:1018C000030C01D1000402E080231B05C918030E9C
:1018D00001D1000202E08023DB04C918030F01D10B
:1018E000000102E080239B04C918830F01D180000E
:1018F00002E080235B04C918002801DB400002E0FD
:1019000080231B04C918803003125918000601D126
:1019100001239943081C00E000207047802108B58E
:10192000C905FFF7CBFF08BD10B543435143C918A4
:10193000040C130C5C43091992B2040C544380B29A
:10194000434350432204240C801861411A041B0CA9
:101950008018594110BD8446830708D18B0706D1F2
:10196000131F04D304C904C0043BFBD21A1D524206
:1019700005D0891A801A8B5C83540132FBD16046F2
:1019800070478446043A09D3830707D109060B0A36
:1019900019430B0C1943043A02C0FCD2043203D0A1
:1019A00001700130013AFBD1604670473743313650
:1019B00031312D393566363132633000001BB700C6
:1019C0000001010000020100000301000004010009
:1019D0000005010000060100000B010100120100DA
:1019E0000013010000000000C0270900900510004E
:1019F000C05C1500F0B31A00200B2000009F2400EB
:101A0000E0322900C0C62D0050973100E067350054
:101A10007038390000093D00401640008023430023
:041A2000C03046008C
:081A24000000803F01000000FA
:0400000300000103F5
:00000001FF
